:100000008CEF0DF00000000098EF0CF000000000F5
:0C001000000000000000000058EF0DF0A0
:10001C006DB409D01F0E6B14016E0150000A03E180
:0A002C00010E006E01D0006A120000
:10003600A49E87C36FFF6DA401D0FDD7A4BE01D0D7
:10004600FDD76BBC02D0006A03D06B84020E006E33
:02005600120096
:100058000301876B886B8851120802E187518E086B
:1000680008E3D8DF005201E004D00301874B882B56
:10007800F2D70301120E885D02E18F0E875D03E35C
:100088007B0E006E05D06B806BA001D0FDD7006A97
:02009800120054
:10009A0089C3F6FF8AC3F7FF8BC3F8FF0900F5CFC0
:1000AA0000F0005218E089C3F6FF8AC3F7FF8BC33A
:1000BA00F8FF0900F5CF00F087C3E1FF88C3E2FF2C
:1000CA0000C0E6FF0301874B882B010E8927000E2B
:1000DA008A238B23DDD787C3E1FF88C3E2FFE66A61
:0200EA00120002
:0400EC006B8412000F
:0A00F0006B826BA201D0FDD7120055
:0E00FA00ADB202D00000FCD787C3AEFF1200EB
:0E010800A8B202D00000FCD769C3A9FF120004
:10011600086A080E0C6E003408360450085ED8B023
:0E01260002D00826D89000360C2EF5D7120015
:1001340091DF13C187F37DDF0301876B7ADF000E44
:10014400006E03016C51005C03E16B510101005D21
:1001540005E200C16BF3000E03016C6F0FD00301C5
:100164006B51800F876F870764DF16D003016B51D3
:10017400C00F876F87075DDF0FD00ED0000E03011D
:100184006A1902E1010E6919EAE0000E6A1902E136
:10019400020E6919EBE0F1D7A9DF13C187F349DF38
:1001A400400E0301876F45DF6BC36FF36CC370F3BD
:1001B4006DC3E9FF6EC3EAFFEE521AE06DC3D9FFC7
:1001C4006EC3DAFFDE50800F0301876F32DF030155
:1001D4006D4B6E2B6F4B702B800E006E800E701962
:1001E400005C03E16F510101005D01E201D0E0D741
:0401F4007BDF12009B
:1001F8000D0E0301876F7DDF0A0E0301876F79DF1C
:020208001200E2
:10020A0026DF13C187F312DF0301876B0FDF020EAC
:10021A000301876F0BDF0BD0800E0301876F06DFA8
:10022A0014D0C00E0301876F01DF0FD00ED0000E6D
:10023A0003016A1902E1010E6919EEE0000E6A195A
:10024A0002E1020E6919EDE0F1D74DDF13C187F320
:10025A00EDDE400E0301876FE9DE03016B6B6C6B09
:10026A00800E6C19006E800E005C04E101010051E1
:10027A0003016B5D07E2A00E876FD8DE03016B4BAB
:10028A006C2BEED730DF13C187F3D0DE0301876B07
:10029A00CDDE0BD0800E0301876FC8DE14D0C00EEE
:1002AA000301876FC3DE0FD00ED0000E03016A1957
:1002BA0002E1010E6919EEE0000E6A1902E1020E6E
:0A02CA006919EDE0F1D70DDF120015
:1002D40003016C6B69C3E9FF6AC3EAFFEECF6BF3FA
:1002E4006B51000A0EE06BC387F305DF03016C2B2F
:1002F4006C516925E96E000E6A21EA6EEECF6BF34C
:04030400EFD712001D
:1003080069C3F6FF6AC3F7FF6BC3F8FF0900F5CFAF
:1003180000F0005211E069C3F6FF6AC3F7FF6BC330
:10032800F8FF0900F5CF87F3E4DE010E0301692722
:0A033800000E6A236B23E4D71200C5
:10034200700E0301876F030E886F6DC389F36EC34E
:100352008AF36FC38BF3A0DE7EDE13C187F36ADEFE
:100362000301876B67DE000E006E03016C51005CB7
:1003720003E16B510101005D05E200C16BF3000E68
:1003820003016C6F0FD003016B51800F876F8707DA
:1003920051DE16D003016B51C00F876F87074ADE0B
:1003A2000FD00ED0000E03016A1902E1010E691985
:1003B200EAE0000E6A1902E1020E6919EBE0F1D7D8
:1003C20096DE13C187F336DE400E0301876F32DEFD
:1003D2006BC385F36CC386F36DC3F6FF6EC3F7FF81
:1003E2006FC3F8FF0900F5CF00F0005222E06DC3A1
:1003F200F6FF6EC3F7FF6FC3F8FF0900F5CF00F0F9
:100402000050800F0301876F15DE010E03016D2777
:10041200000E6E236F23854B862B800E006E800E9E
:100422008619005C03E185510101005D01E201D002
:06043200D3D75BDE1200CF
:100438003C0E7B6EAF0E7A6E0301526B536B798064
:08044800A192A292A082120011
:1004500003DE13C187F3EFDD0301876BECDD800E54
:10046000006E800E03016C19005C03E16B51010109
:10047000005D05E200C16BF3000E03016C6F0FD04D
:1004800003016B51800F876F8707D5DD16D00301FD
:100490006B51C00F876F8707CEDD0FD00ED0000ED7
:1004A00003016A1902E1010E6919EAE0000E6A19F6
:1004B00002E1020E6919EBE0F1D71ADE13C187F3EE
:1004C000BADD400E0301876FB6DD03016D51800F69
:0804D000876FB1DD0BDE1200A5
:0E04D800570E0D6E0D2EFED700000000120014
:1004E600520E0301546F020E556F83DE5D0E03013B
:1004F600696F2B0E6A6F000E6B6F03DF520E0301DE
:10050600696F020E6A6FE3DE74DE0201616B010E33
:100516000301696F000E6A6F75DE010E0301696FD4
:10052600000E6A6F010E6B6F000E6C6F520E6D6FD0
:10053600020E6E6FFCDD020E0301696F000E6A6F1C
:10054600010E6B6F000E6C6FD10E6D6F290E6E6F04
:10055600000E6F6FF3DE000E0301531902E1000E69
:10056600521922E101013B4B3C2B020E0301696F3C
:10057600000E6A6F090E6B6F000E6C6F300E010174
:100586003B2503016D6F61DF3D0E0B6EE10E0C6EB8
:100596003F0E0D6E0D2EFED70C2EFCD70B2EFAD766
:1005A600000000008C9801D08C88830E0301696FCF
:1005B6002B0E6A6F000E6B6FA4DE300E01013B2519
:1005C6000301876F97DD15DE070E0B6E170E0C6E97
:1005D6006A0E0D6E0D2EFED70C2EFCD70B2EFAD7FB
:0E05E60000000F0E536E000E546E23DF120045
:1005F40067C301F068C302F0010E0301675F000ED8
:10060400685B000E021802E1000E01181FE063C3CC
:10061400E9FF64C3EAFF65C3D9FF66C3DAFFEE509E
:10062400DE180FE063C3E9FF64C3EAFF65C3D9FFC3
:1006340066C3DAFFDE50EE5C006E016A000E015AFA
:1006440007D0634B642B654B662BD2D7006A016AD3
:02065400120092
:100656004D6A4E6A010E4E5C02E1000E4D5C0AE2E6
:10066600520E4D24E16E020E4E20E26EE66A4D4AAF
:100676004E2AF0D74F6A506A4D6A4E6AA4AA02D033
:0E068600AACF4CF04C6A516A526AA38A120045
:1006940063C3F6FF64C3F7FF65C3F8FF0900F5CF32
:1006A40000F0005211E063C3F6FF64C3F7FF65C3B3
:1006B400F8FF0900F5CF69F325DD010E0301632777
:0A06C400000E64236523E4D7120042
:1006CE00086A096A100E0C6E013408360936045099
:1006DE00085E0550D8A0053C095ED8B007D004507E
:1006EE0008260550D8B0053C0926D89000360136AC
:0606FE000C2EEAD71200E9
:1007040063C302F064C303F002C000F003C001F04D
:10071400024A032A00C0E9FF01C0EAFFEE5201E0E9
:10072400F3D703016351025C006E64510358016EF8
:0A073400010E005E000E015A1200D3
:10073E000301666B030E665D0AE266516425E16E87
:10074E00000E6521E26E200EE66E662BF3D7665123
:10075E006425E16E000E6521E26EE66A660766515B
:10076E006425676F000E6521686F0A0E046E63C301
:10077E0000F0CADC08C000F0300E002667C3E1FFAF
:10078E0068C3E2FF00C0E6FF0A0E046E63C300F00A
:10079E00BBDC00C063F30050000A01E102D0660723
:0407AE00DED7120080
:1007B2007A0E0301696F2A0E6A6F000E6B6FA3DD5A
:1007C20058C363F35A0E0301646F030E656FB6DFFD
:1007D2005A0E696F030E6A6F7CDD8C0E696F2B0EE9
:1007E2006A6F000E6B6F8FDD710E0301696F2B0E46
:1007F2006A6F000E6B6F87DD2EDC58C387F31ADC3D
:1008020000C059F30050000A0BE0D40E0301696FD7
:100812002A0E6A6F000E6B6F76DD0301596B0BD0E7
:100822000301670E696F2B0E6A6F000E6B6F6BDD33
:10083200010E0301596F59DCDEDC59C300F01200CE
:1008420003015A6B5B6B1F0E0B6E710E0C6E1E0E4C
:100852000D6E0D2EFED70C2EFCD70B2EFAD70000F4
:100862002CEC00F013C187F31BEC00F000C058F32E
:10087200000E0301596F000E591902E1000E5819BA
:1008820005E05AC300F05BC301F0E0D05A4B5B2B8A
:100892000D0E0B6E2D0E0C6ED70E0D6E0D2EFED79D
:1008A2000C2EFCD70B2EFAD700000000876B1BEC36
:1008B20000F000C058F3000E0301596F800E006E65
:1008C200800E5919005C02E15851000805E25AC332
:1008D20000F05BC301F0BAD05A4B5B2B240E876F3A
:1008E2001BEC00F00C0E0301876F1BEC00F0060EF0
:1008F2000301876F1BEC00F0250E0301876F1BECD1
:1009020000F0060E0301876F1BEC00F0110E0301CD
:10091200876F1BEC00F0420E0301876F1BEC00F0A7
:10092200960E0301876F1BEC00F0240E0301876F04
:100932001BEC00F000C058F3000E0301596F800E4B
:10094200006E800E5919005C02E15851000805E260
:100952005AC300F05BC301F079D05A4B5B2B0C0EEB
:10096200876F1BEC00F000C058F3000E0301596FB3
:10097200800E006E800E5919005C02E15851000889
:1009820005E25AC300F05BC301F060D05A4B5B2B07
:10099200060E876F1BEC00F000C058F3000E030137
:1009A200596F800E006E800E5919005C02E1585199
:1009B200000805E25AC300F05BC301F047D05A4B6E
:1009C2005B2B020E876F1BEC00F000C058F3000E89
:1009D2000301596F800E006E800E5919005C02E10E
:1009E2005851000805E25AC300F05BC301F02ED053
:1009F2005A4B5B2B010E876F1BEC00F000C058F3C3
:100A0200000E0301596F800E006E800E5919005CB2
:100A120002E15851000805E25AC300F05BC301F03D
:100A220015D0070E0B6E170E0C6E6A0E0D6E0D2E84
:100A3200FED70C2EFCD70B2EFAD7000076EC00F076
:0E0A42005A4B5B2B5AC300F05BC301F012004D
:100A500058C304F059C305F003015C515D1124E053
:100A6000010E5C5F000E5D5B04C002F005C003F088
:100A7000044A052A5AC300F05BC301F05A4B5B2BB2
:100A800000C0E9FF01C0EAFF02C0E1FF03C0E2FFCE
:100A9000EECFE6FF02C0E9FF03C0EAFFEECF00F0B1
:100AA000005201E101D0D8D75CC300F05DC301F072
:100AB000010E5C5F000E5D5B0050011008E004C099
:100AC000E1FF05C0E2FFE66A044A052AEDD758C3F4
:080AD00000F059C301F012000F
:100AD80003015C6B050E5C5D0AE25C515A25E16E10
:100AE800000E5B21E26E200EE66E5C2BF3D75C51A4
:100AF8005A25E16E000E5B21E26EE66A5C075C51E6
:100B08005A255D6F000E5B215E6F0A0E046E000EA3
:100B1800056E58C300F059C301F0D5DD08C000F0D8
:100B280009C001F0300E00265DC3E1FF5EC3E2FF9D
:100B380000C0E6FF0A0E046E000E056E58C300F0F2
:100B480059C301F0C0DD00C058F301C059F3000ECD
:100B5800011802E1000E001801E102D05C07CFD7AE
:020B6800120079
:100B6A00150E7B6E9F0E7A6E0301526B536B799250
:100B7A00798A7988799C79967994798E7990A292F2
:060B8A00A192A0921200EE
:100B9000FD0EC16EFF0EC26EFF0E926E9294FF0E9E
:100BA000936EFF0E956EFF0E946EFF0E986E959CE1
:100BB000958E9986959896988C988D989594938211
:020BC000120021
:100BC2000900F5CFE6FF0006FBE10106F9E112009C
:100BD200FA0E0101476F000E486F870E496F030E30
:100BE2004A6FFF0E4B6FFF0E4C6F000E4D6F000EE3
:100BF2004E6FFF0E436FFF0E446F000E456F000EE7
:100C0200466FFF0E3D6FFF0E3E6F000E3F6F000EF0
:100C1200406FAD8A900EAC6E948E949C9EAA03D0C7
:080C2200AFCF00F0FBD7120078
:100C2A00959A959C8C9A8C9C958A958C6D9E6D9CB8
:060C3A00380E6C6E120082
:100C4000080E0101476F010E486F690E496F030ED0
:100C50004A6FFF0E4B6FFF0E4C6F000E4D6F000E74
:100C60004E6FFF0E436FFF0E446F000E456F000E78
:100C7000466FFF0E3D6FFF0E3E6F000E3F6F000E82
:100C8000406FA88A900E9C6E98849892A4AA03D074
:080C9000AACF00F0FBD712000F
:100C980058C304F059C305F004C0E9FF05C0EAFFD2
:100CA800EE5203E0044A052AF7D704C002F005C053
:100CB80003F0044A052A5AC300F05BC301F003019C
:100CC8005A4B5B2B00C0E9FF01C0EAFF02C0E1FFFD
:100CD80003C0E2FFEECFE6FF02C0E9FF03C0EAFF70
:100CE800EE5201E0E2D758C300F059C301F01200F8
:100CF800C26A070EC16EC18E58C300F0003600905C
:100D0800003600900050C212C2806CEC02F0C28221
:100D1800C2A201D0FDD7C4CF01F0006AC3500012AF
:080D2800000E0112C29012003E
:100D300003015B6B58C3E9FF59C3EAFFEECF5AF3D7
:100D40005A51000A0FE05AC369F384EC00F0030122
:100D50005B2B5B515825E96E000E5921EA6EEECFF0
:060D60005AF3EED7120069
:100D66005CC300F003015C07005228E058C3E9FFAA
:100D760059C3EAFFEE50000A0CE058C3E9FF59C315
:100D8600EAFF5AC3D9FF5BC3DAFFEE50DE1801E172
:100D96000FD058C3E9FF59C3EAFF5AC3D9FF5BC353
:100DA600DAFFDE50EE5C006E016A000E015A08D0D2
:100DB6000301584B592B5A4B5B2BD2D7006A016A59
:020DC600120019
:100DC80003015A6B5B6BEE0E696F280E6A6F000E9B
:100DD8006B6F84EC01F0010E03015E6F000E5F6F14
:100DE800520E636F020E646F89DC00C05CF301C0B1
:100DF8005DF3070E586F000E596F800E5919006E7B
:100E0800800E5D19005C02E15C51585DD8B0ECD0F1
:100E1800C6D0520E5825E96E020E5921EA6EEE50E0
:100E28002C0A0EE1070E5A25E16E010E5B21E26ED7
:100E3800E66A5A6B5B6B020E5E6F000E5F6FD1D075
:100E4800070E5A25E16E010E5B21E26E520E5825FF
:100E5800E96E020E5921EA6EEECFE6FF5A4B5B2B84
:100E6800C0D0520E5825E96E020E5921EA6EEE5096
:100E78002C0A0EE1140E5A25E16E010E5B21E26E7A
:100E8800E66A5A6B5B6B030E5E6F000E5F6FA9D04C
:100E9800140E5A25E16E010E5B21E26E520E5825A2
:100EA800E96E020E5921EA6EEECFE6FF5A4B5B2B34
:100EB80098D0520E5825E96E020E5921EA6EEE506E
:100EC8002C0A0EE12F0E5A25E16E010E5B21E26E0F
:100ED800E66A5A6B5B6B040E5E6F000E5F6F81D023
:100EE8002F0E5A25E16E010E5B21E26E520E582537
:100EF800E96E020E5921EA6EEECFE6FF5A4B5B2BE4
:100F080070D0520E5825E96E020E5921EA6EEE5045
:100F18002C0A07E15A6B5B6B050E5E6F000E5F6F64
:100F280060D0230E5A25E16E010E5B21E26E520E4F
:100F38005825E96E020E5921EA6EEECFE6FF5A4BAC
:100F48005B2B4FD0520E5825E96E020E5921EA6EDE
:100F5800EE502C0A0EE11F0E5A25E16E010E5B21A0
:100F6800E26EE66A5A6B5B6B080E5E6F000E5F6F8F
:100F780038D01F0E5A25E16E010E5B21E26E520E2B
:100F88005825E96E020E5921EA6EEECFE6FF5A4B5C
:100F98005B2B27D05CC358F35DC359F322D0000EF6
:100FA8005F1902E1010E5E19D8B433D7000E5F193C
:100FB80002E1020E5E19D8B454D7000E5F1902E19F
:100FC800030E5E19D8B475D7000E5F1902E1040E3E
:100FD8005E1997E0000E5F1902E1050E5E19B2E096
:100FE800D9D7584B592B09D7FCEC00F0BF0E030199
:100FF800696F2B0E6A6F000E6B6F84EC01F0070EA1
:101008000301696F010E6A6F6AEC01F0090E876FC0
:101018007DEC00F0B20E0301696F2B0E6A6F000EB3
:101028006B6F84EC01F02F0E0301696F010E6A6F7C
:101038006AEC01F0090E876F7DEC00F0470E0301A2
:10104800696F2B0E6A6F000E6B6F84EC01F0140E43
:101058000301696F010E6A6F6AEC01F0090E876F70
:101068007DEC00F0090E0301696F2B0E6A6F000E0C
:101078006B6F84EC01F01F0E0301696F010E6A6F3C
:101088006AEC01F0090E876F7DEC00F0FCEC00F0D3
:0A1098005EC300F05FC301F0120018
:1010A2000301566B576B010E575D02E1000E565D50
:1010B2000AE24F0E5625E16E010E5721E26EE66AF4
:1010C200564B572BF0D70101416B426B0301566B14
:1010D200576B9EAA02D0AFCF4FF202014F6B506BFB
:0610E200516BA08A120010
:1010E800020E0301696F000E6A6F05EC01F0010E34
:0E10F8000301696F000E6A6F05EC01F0120033
:10110600C29EC29CC29AC298C296C284C280FF0E78
:10111600C16EC192C18EC19CC18AC188C196C1826D
:06112600C194C19012000B
:10112C005AC304F05BC305F058C302F059C303F073
:10113C005CC300F05DC301F0010E03015C5F000EA7
:10114C005D5B005001100FE004C0E9FF05C0EAFF31
:10115C0002C0E1FF03C0E2FFEECFE6FF024A032A22
:10116C00044A052AE5D758C300F059C301F0120010
:10117C00010E0301696F000E6A6F010E6B6F000E9A
:10118C006C6F9E0E6D6F290E6E6F000E6F6FA1EC63
:10119C0001F0020E0301696F000E6A6F010E6B6F96
:1011AC00000E6C6FAF0E6D6F290E6E6F000E6F6FB1
:1011BC00A1EC01F01F0E0B6E710E0C6E1E0E0D6E5F
:1011CC000D2EFED70C2EFCD70B2EFAD700008C98C8
:1011DC008D98CA0E0301696F2B0E6A6F000E6B6F30
:1011EC0084EC01F0C50E0301636F2B0E646F000ECF
:1011FC00656F4AEC03F01F0E0B6E710E0C6E1E0E1B
:10120C000D6E0D2EFED70C2EFCD70B2EFAD7000030
:10121C0001013B6B3C6B320E536E000E546E1CEC9A
:10122C0002F02F0E696F290E6A6F000E6B6F84EC43
:10123C0001F02BEC03F0240E0301696F84EC00F039
:10124C004E0E0C6EEB0E0D6E0D2EFED70C2EFCD72B
:10125C00240E0301696F84EC00F04E0E0C6EEB0E45
:10126C000D6E0D2EFED70C2EFCD7240E0301696FCC
:10127C0084EC00F04E0E0C6EEB0E0D6E0D2EFED7A8
:10128C000C2EFCD7000E521802E1000E51180EE184
:10129C00000E0301531902E1000E521907E1000E72
:1012AC00505C02E1030E4F5C01E2ECD70301520EDD
:1012BC00636F020E646F340E656F000E666F030E63
:1012CC00676F000E686FFAEC02F0000E011802E175
:1012DC00000E001808E0000E0301531902E1000E85
:1012EC00521901E1A6D773EC02F0DD0E696F270EDF
:1012FC006A6F000E6B6F84EC01F02BEC03F0FC0EAC
:10130C000301636F2A0E646F000E656F4AEC03F0E5
:10131C000D0E0301696F84EC00F01F0E0B6E710E45
:10132C000C6E1E0E0D6E0D2EFED70C2EFCD70B2E3A
:10133C00FAD70000000E521802E1000E51180EE10F
:10134C00000E0301531902E1000E521907E1000EC1
:10135C00505C02E1030E4F5C01E2ECD70301520E2C
:10136C00636F020E646F400E656F000E666F030EA6
:10137C00676F000E686FFAEC02F0000E011802E1C4
:10138C00000E001808E0000E0301531902E1000ED4
:10139C00521901E1B2D773EC02F0560E696F290EA7
:1013AC006A6F000E6B6F84EC01F02BEC03F09C0E5B
:1013BC000301636F2B0E646F000E656F4AEC03F034
:1013CC000D0E0301696F84EC00F01F0E0B6E710E95
:1013DC000C6E1E0E0D6E0D2EFED70C2EFCD70B2E8A
:1013EC00FAD70000000E521802E1000E51180EE15F
:1013FC00000E0301531902E1000E521907E1000E11
:10140C00505C02E1030E4F5C01E2ECD70301520E7B
:10141C00636F020E646F3C0E656F000E666F030EF9
:10142C00676F000E686FFAEC02F0000E011802E113
:10143C00000E001808E0000E0301531902E1000E23
:10144C00521901E1B2D773EC02F06C0E696F280EE1
:10145C006A6F000E6B6F84EC01F02BEC03F0AB0E9B
:10146C000301636F2B0E646F000E656F4AEC03F083
:10147C000D0E0301696F84EC00F01F0E0B6E710EE4
:10148C000C6E1E0E0D6E0D2EFED70C2EFCD70B2ED9
:10149C00FAD70000000E521802E1000E51180EE1AE
:1014AC00000E0301531902E1000E521907E1000E60
:1014BC00505C02E1030E4F5C01E2ECD70301520ECB
:1014CC00636F020E646F380E656F000E666F030E4D
:1014DC00676F000E686FFAEC02F0000E011802E163
:1014EC00000E001808E0000E0301531902E1000E73
:1014FC00521901E1B2D773EC02F0A90E696F2A0EF2
:10150C006A6F000E6B6F84EC01F02BEC03F0D90EBC
:10151C000301636F2B0E646F000E656F4AEC03F0D2
:10152C000D0E0301696F84EC00F01F0E0B6E710E33
:10153C000C6E1E0E0D6E0D2EFED70C2EFCD70B2E28
:10154C00FAD70000000E521802E1000E51180EE1FD
:10155C00000E0301531902E1000E521907E1000EAF
:10156C00505C02E1030E4F5C01E2ECD70301520E1A
:10157C00636F020E646F280E656F000E666F030EAC
:10158C00676F000E686FFAEC02F0000E011802E1B2
:10159C00000E001808E0000E0301531902E1000EC2
:1015AC00521901E1B2D773EC02F07F0E696F270E6E
:1015BC006A6F000E6B6F84EC01F02BEC03F0D40E11
:1015CC000301636F2B0E646F000E656F4AEC03F022
:1015DC000D0E0301696F84EC00F01F0E0B6E710E83
:1015EC000C6E1E0E0D6E0D2EFED70C2EFCD70B2E78
:1015FC00FAD70000000E521802E1000E51180EE14D
:10160C00000E0301531902E1000E521907E1000EFE
:10161C00505C02E1030E4F5C01E2ECD70301520E69
:10162C00636F020E646F240E656F000E666F030EFF
:10163C00676F000E686FFAEC02F0000E011802E101
:10164C00000E001808E0000E0301531902E1000E11
:10165C00521901E1B2D773EC02F081B209D09F0E9E
:10166C00696F270E6A6F000E6B6F84EC01F009D066
:10167C00190E0301696F280E6A6F000E6B6F84ECF4
:10168C0001F02BEC03F081B220D08A0E0301636FC2
:10169C002A0E646F000E656F4AEC03F00D0E030109
:1016AC00696F84EC00F0020E0301696F000E6A6F23
:1016BC00010E6B6F000E6C6F370E6D6F2A0E6E6F16
:1016CC00000E6F6FA1EC01F01FD06A0E0301636F67
:1016DC002A0E646F000E656F4AEC03F00D0E0301C9
:1016EC00696F84EC00F0020E0301696F000E6A6FE3
:1016FC00010E6B6F000E6C6F260E6D6F2A0E6E6FE7
:10170C00000E6F6FA1EC01F01F0E0B6E710E0C6EC4
:10171C001E0E0D6E0D2EFED70C2EFCD70B2EFAD7EF
:10172C000000000E521802E1000E51180EE1000EDE
:10173C000301531902E1000E521907E1000E505C2F
:10174C0002E1030E4F5C01E2ECD70301520E636F12
:10175C00020E646F200E656F000E666F030E676FCE
:10176C00000E686FFAEC02F0000E011802E1000E98
:10177C00001808E0000E0301531902E1000E521983
:10178C0001E17FD773EC02F0320E536E000E546EF3
:10179C00430E696F290E6A6F000E6B6F84EC01F0BB
:1017AC002BEC03F0CF0E0301636F2B0E646F000E56
:1017BC00656F4AEC03F00D0E0301696F84EC00F0C9
:1017CC00040E0B6E0C0E0C6E330E0D6E0D2EFED722
:1017DC000C2EFCD70B2EFAD700000000000E52186E
:1017EC0002E1000E51180EE1000E0301531902E143
:1017FC00000E521907E1000E505C02E1030E4F5C23
:10180C0001E2ECD70301520E636F020E646F2C0ED3
:10181C00656F000E666F030E676F000E686FFAEC53
:10182C0002F0000E011802E1000E001808E0000E94
:10183C000301531902E1000E521901E1B1D773EC07
:10184C0002F03D0E0B6EE10E0C6E3F0E0D6E0D2E6A
:10185C00FED70C2EFCD70B2EFAD700000000320E50
:10186C00536E000E546E1CEC02F0870E696F280E3E
:10187C006A6F000E6B6F84EC01F02BEC03F0DE0E44
:10188C000301636F2B0E646F000E656F4AEC03F05F
:10189C000D0E0301696F84EC00F01F0E0B6E710EC0
:1018AC000C6E1E0E0D6E0D2EFED70C2EFCD70B2EB5
:1018BC00FAD70000000E521802E1000E51180EE18A
:1018CC00000E0301531902E1000E521907E1000E3C
:1018DC00505C02E1030E4F5C01E2ECD70301520EA7
:1018EC00636F020E646F300E656F000E666F030E31
:1018FC00676F000E686FFAEC02F0000E011802E13F
:10190C00000E001808E0000E0301531902E1000E4E
:10191C00521901E1B2D773EC02F03BC100F03CC1AB
:04192C0001F01200B4
:1019300000C01BF001C01AF0E1CF1EF0E2CF1FF093
:10194000E9CF1CF0EACF1DF09EAA4BD09DAA49D04A
:10195000ACA203D0AC98AC88AC92ACA402D0AFCF10
:101960004FF2AFCF4FF202014F510D0A08E0010EC6
:101970000301575D02E1000E565D01E223D0010E26
:101980000201506F000E516F010E0301575D02E11D
:10199000000E565D05E3020E0201506F000E516FFE
:1019A000A09A4F0E03015625E16E010E5721E26EFB
:1019B000E66A56C341F157C342F1566B576B0201B9
:1019C0004F6B0FD04F0E03015625E16E010E5721CC
:1019D000E26E4FC2E6FF56C341F157C342F1564B88
:1019E000572BA4AA58D0A3AA56D09CA202D09C9848
:1019F0009C889CA402D0AACF4CF0AACF4CF0000E39
:101A00004E5C02E1FF0E4D5C08E244500D0A04E119
:101A10004C500D0A01E101D030D0A39A010E4D5C6B
:101A2000006E000E4E58016E520E0024E96E020E3A
:101A30000120EA6EEE500A0A0DE1010E4D5C006EC7
:101A4000000E4E58016E520E0024E16E020E01206F
:101A5000E26EE66A520E4D24E16E020E4E20E26EF8
:101A6000E66A4DC04FF04EC050F04D6A4E6A4C6A67
:101A7000010E516E000E526E0ED0520E4D24E16ECC
:101A8000020E4E20E26E4CC0E6FF4DC04FF04EC03D
:101A900050F04D4A4E2A1BC000F01AC001F01CC085
:101AA000E9FF1DC0EAFF1EC0E1FF1FC0E2FF1100F9
:101AB00000C019F001C018F0156ED8CF16F0E0CFB5
:101AC00017F0A0A21ED0A1A21CD0010E535C006E84
:101AD000000E5458016E00C053F001C054F0000EC7
:101AE000541802E1000E53180BE1010E0301526F6E
:101AF000000E536F7990150E7B6E9F0E7A6EA0923A
:101B0000A1921750E06E1650D86E153A153819C0CC
:081B100000F018C001F0100004
:101B1800F1EC15F0D38CD38AD388D382D3909B6A07
:101B28009B8CD3B601D0FDD7C8EC05F08C94140E6D
:101B3800536E000E546E7F0E0101016F000E026F8E
:101B480000017F6B576A020E0A6E310E0B6E620E31
:101B58000C6E450E0D6E0D2EFED70C2EFCD70B2EDF
:101B6800FAD70A2EF8D77E86010E7F6E370EB06E32
:101B7800AD84E9EC05F00C0E0301876F7DEC00F0F5
:101B88001F0E0B6E710E0C6E1E0E0D6E0D2EFED7F7
:101B98000C2EFCD70B2EFAD700005A0E0301696FE2
:101BA800260E6A6F000E6B6F84EC01F0680E03015D
:101BB800696F250E6A6F000E6B6F84EC01F01F0EC3
:101BC8000301696F250E6A6F000E6B6F84EC01F0DC
:101BD800360E0301696F270E6A6F000E6B6F84EC77
:101BE80001F0240E0301696F260E6A6F000E6B6FF9
:101BF80084EC01F0BF0E0301696F270E6A6F000EB7
:101C08006B6F84EC01F0AC0E0301696F250E6A6FEF
:101C1800000E6B6F84EC01F0EC0E0301696F250E6A
:101C28006A6F000E6B6F84EC01F0E50E0301696FBB
:101C3800260E6A6F000E6B6F84EC01F00D0E0B6EB2
:101C48002D0E0C6ED70E0D6E0D2EFED70C2EFCD75A
:101C58000B2EFAD7000000007C86020E7D6E700EF7
:101C6800AB6EA88420EC06F00D0E0B6E2D0E0C6EDC
:101C7800D70E0D6E0D2EFED70C2EFCD70B2EFAD7D5
:101C8800000000001E0E6E6E15EC06F0350E030106
:101C9800696F280E6A6F000E6B6F84EC01F0780E86
:101CA800536E000E546EB5EC05F0740E0101136FFF
:101CB800740E0001FF6F100E0101006F5C0E03012E
:101CC800696F270E6A6F000E6B6F84EC01F0FFC01E
:101CD80058F3D9EC03F000C005F1000E0101066FBE
:101CE800FCEC00F01A0E0301696F290E6A6F000EF2
:101CF8006B6F84EC01F021EC04F000C005F101C029
:101D080006F10A0E0B6E220E0C6EA10E0D6E0D2E34
:101D1800FED70C2EFCD70B2EFAD774EC08F00A0E5F
:101D28000B6E220E0C6EA10E0D6E0D2EFED70C2E14
:101D3800FCD70B2EFAD7010E0301696F000E6A6FEC
:101D4800010E6B6F000E6C6F590E6D6F2A0E6E6F61
:101D5800000E6F6FA1EC01F0020E0301696F000E17
:101D68006A6F010E6B6F000E6C6F480E6D6F2A0E56
:101D78006E6F000E6F6FA1EC01F07A0E0B6EC10E44
:101D88000C6E810E0D6E0D2EFED70C2EFCD70B2E71
:101D9800FAD70000000051EC08F0E20E0301696F69
:101DA8002A0E6A6F000E6B6F84EC01F083EC08F06A
:101DB800020E0301696F000E6A6F010E6B6F000E51
:101DC8006C6F150E6D6F2A0E6E6F000E6F6FA1ECA3
:101DD80001F07A0E0B6EC10E0C6E810E0D6E0D2E7B
:101DE800FED70C2EFCD70B2EFAD700000000D50E1C
:101DF8000301696F280E6A6F000E6B6F84EC01F0A7
:101E080051EC08F02BEC03F08C94020E0301696F7F
:101E1800000E6A6F05EC01F0010E0301696F000EF8
:101E28006A6F010E6B6F000E6C6FC00E6D6F290E1E
:101E38006E6F000E6F6FA1EC01F05C0E0B6E510E11
:101E48000C6E600E0D6E0D2EFED70C2EFCD70B2ED1
:101E5800FAD700009D8AA38AF28CF28ED08E0101F7
:101E6800036B046B446A8C840D0E0B6E2D0E0C6E86
:101E7800D70E0D6E0D2EFED70C2EFCD70B2EFAD7D3
:101E8800000000008C940D0E0B6E2D0E0C6ED70EFC
:101E98000D6E0D2EFED70C2EFCD70B2EFAD7000098
:101EA80000008C840D0E0B6E2D0E0C6ED70E0D6E71
:101EB8000D2EFED70C2EFCD70B2EFAD700000000F3
:101EC800BEEC08F000C005F101C006F1FB0E696F19
:101ED800270E6A6F000E6B6F84EC01F005C158F392
:101EE80006C159F3570E03015A6F000E5B6F6CEC75
:101EF80005F0570E696F000E6A6F6AEC01F0000E6C
:101F08000101061902E1090E05190AE13C0E030157
:101F1800696F2B0E6A6F000E6B6F84EC01F009D0AD
:101F2800690E0301696F290E6A6F000E6B6F84ECEE
:101F380001F0FCEC00F0020E0301696F000E6A6FFD
:101F480005EC01F0000E0101061902E1090E051960
:101F580012E1020E0301696F000E6A6F010E6B6FCA
:101F6800000E6C6F040E6D6F2A0E6E6F000E6F6F91
:101F7800A1EC01F011D0020E0301696F000E6A6F27
:101F8800010E6B6F000E6C6FF30E6D6F290E6E6F86
:101F9800000E6F6FA1EC01F07A0E0B6EC10E0C6E85
:101FA800810E0D6E0D2EFED70C2EFCD70B2EFAD7F8
:101FB8000000000051EC08F02BEC03F00D0E446E0D
:101FC800640E536E000E546E1CEC02F07F0E01017D
:101FD800016F000E026F01C187F302C188F3A20EE0
:101FE8000301896F280E8A6F000E8B6F4DEC00F08D
:101FF800040E01010125E16E000E0221E26E006A65
:1020080083BE002A300E002600C0E6FF0D0E012513
:10201800E16E000E0221E26E006A87B6002A300ED9
:10202800002600C0E6FF010E0301586F7CEC06F0A5
:1020380000C055F001C056F000C058F301C059F374
:10204800570E03015A6F000E5B6F6CEC05F001C16F
:1020580058F302C159F3570E5A6F000E5B6F4CECE0
:1020680006F001C169F302C16AF36AEC01F0FCEC05
:1020780000F001C158F302C159F398EC06F00D0EB7
:10208800696F84EC00F02BEC03F074EC08F001C1EC
:1020980087F302C188F3520E0301896F2B0E8A6FF2
:1020A800000E8B6F4DEC00F0030E01010125E16E6F
:1020B800000E0221E26E006A83BE002A300E00265E
:1020C80000C0E6FF080E0125E16E000E0221E26E57
:1020D800006A87B6002A300E002600C0E6FF01C15C
:1020E80058F302C159F3570E03015A6F000E5B6F84
:1020F8004CEC06F0010E696F000E6A6F010E6B6FF3
:10210800000E6C6F01C16DF302C16EF39AEC00F022
:10211800020E0301696F000E6A6F010E6B6F000EED
:102128006C6FE20E6D6F290E6E6F000E6F6FA1EC73
:1021380001F03D0E0B6EE10E0C6E3F0E0D6E0D2E76
:10214800FED70C2EFCD70B2EFAD700000000000E8D
:102158000301531902E1000E521907E1000E52184B
:1021680002E1000E511801E1F2D7000E521802E107
:10217800010E5118D8A424D103019A0E696F2A0EB2
:102188006A6F000E6B6F84EC01F0520E0301696FE9
:10219800020E6A6F6AEC01F0FCEC00F0570E0301C6
:1021A800876F000E886F940E896F2B0E8A6F000E52
:1021B8008B6F4DEC00F0520E0301586F020E596FF1
:1021C800570E5A6F000E5B6F070E5C6FB3EC06F08C
:1021D800000E011802E1000E0018D8A4EDD0E4ECBE
:1021E80006F000C04AF001C04BF0000E011802E1F1
:1021F800050E0018D8A4E0D0040E0301696F290E5B
:102208006A6F000E6B6F84EC01F0020E0301696FB8
:10221800000E6A6F05EC01F0570E0301876F000E80
:10222800886F8D0E896F290E8A6F000E8B6F4DECAB
:1022380000F0070E0301636F010E646F82EC03F078
:1022480000C005F101C006F15B0E586F000E596F12
:10225800070E5A6F010E5B6F00C05CF301C05DF39F
:1022680096EC08F00001676B020E0301696F000E1F
:102278006A6F010E6B6F000E6C6F570E6D6F000E5C
:102288006E6F9AEC00F0070E0301696F010E6A6F1A
:102298006AEC01F0FCEC00F05C0E0B6E510E0C6E5B
:1022A800600E0D6E0D2EFED70C2EFCD70B2EFAD716
:1022B8000000570E0301876F000E886FB90E896FF3
:1022C8002B0E8A6F000E8B6F4DEC00F02F0E030162
:1022D800636F010E646F82EC03F000C005F101C06A
:1022E80006F15C0E586F000E596F2F0E5A6F010ED3
:1022F8005B6F00C05CF301C05DF396EC08F0000171
:10230800676B010E0301696F000E6A6F010E6B6F38
:10231800000E6C6F570E6D6F000E6E6F9AEC00F02A
:10232800570E0301876F000E886F7C0E896F290E88
:102338008A6F000E8B6F4DEC00F0140E0301636F73
:10234800010E646F82EC03F000C005F101C006F1D4
:102358005C0E586F000E596F140E5A6F010E5B6FAA
:1023680000C05CF301C05DF396EC08F00001676BF8
:10237800020E0301696F000E6A6F05EC01F0020E90
:102388000301696F000E6A6F010E6B6F000E6C6FB0
:10239800570E6D6F000E6E6F9AEC00F0B70E0B6E55
:1023A800A10E0C6EC30E0D6E0D2EFED70C2EFCD793
:1023B8000B2EFAD7000000002BEC03F051EC08F0CC
:1023C8000201000E511902E1010E501970E12BECC7
:1023D80003F0B80E0301696F2A0E6A6F000E6B6F67
:1023E80084EC01F04F0E0301696F010E6A6F6AEC0D
:1023F80001F0FCEC00F074EC08F0570E0301586F84
:10240800000E596F4F0E5A6F010E5B6F100E5C6F06
:10241800000E5D6F28EC05F0010E696F000E6A6F03
:10242800010E6B6F000E6C6FC60E6D6F2A0E6E6F0D
:10243800000E6F6FA1EC01F0020E0301696F000E30
:102448006A6F010E6B6F000E6C6F570E6D6F000E8A
:102458006E6F9AEC00F03D0E0B6EE10E0C6E3F0EA7
:102468000D6E0D2EFED70C2EFCD70B2EFAD70000C2
:1024780000004F0E0301586F010E596F450E5A6F39
:10248800000E5B6F040E5C6FB3EC06F0000E0118D3
:1024980002E1000E00180BE1530E0301586F010E04
:1024A800596F98EC06F051EC08F02BEC03F051EC66
:1024B80008F02BEC03F0000E0201511902E1020EA4
:0C24C800501902E151EC08F07BD5FFD761
:102BE20010EE20F02C0E006E010E016EB90EF66E84
:0E2BF200260EF76E000EF86EE1EC05F01200F4
:1024D40050726F6A6574203A20436C69636B65724D
:1024E400325F31384638374A35305F524E34315FC7
:1024F40042545F6D61697472655F4C43443231319B
:10250400395F4750535F416E64726F69645F323064
:0B25140031362E6D637070690D0A00F7
:10251F0020536F75726365204D696B726F43204353
:10252F006C69636B6572325F31384638374A3530C4
:10253F005F524E34315F4750535F53746172616421
:10254F00696374325F4C43445F4849445F5F31367F
:09255F00303830352E630D0A00FE
:10256800204469726563746F7279203A433A5F4D0B
:10257800696B726F435F4D657350726F6A657473F0
:102588005F4D696B726F435F31384638374A353073
:102598005F524E34315F4750535F416E64726F69CA
:0425A800640D0A00B4
:1025AC00205541525432203139323030206264731C
:1025BC0020436C69636B657232204D696B726F429C
:1025CC007573233120203C2D3E20426C7565546F71
:1025DC006F7468436C69636B20524E34310D0A0082
:1025EC00205472616D652047505320656D69736589
:1025FC00207061722053746172616469637432205B
:10260C0076696120426C7565546F6F7468202D3E3D
:08261C00524E3431200D0A007A
:1026240020554152543120333834303020626473A1
:1026340020436C69636B657232204D696B726F6203
:102644007573233220203C2D3E207465726D696EB3
:06265400616C200D0A007C
:10265A002048617264776172653A20436C69636BE2
:10266A006572322031384638374A3530202B2042BD
:10267A006C7565546F6F746820436C69636B0D0ADF
:01268A00004F
:10268B0054657374732049542055415254312C5561
:10269B00415254322C54696D6572302C4144433095
:0E26AB00202620425420524E34310D0A2000C9
:0426B900414F4B0042
:0426BD00414F4B003E
:0426C100414F4B003A
:0426C500414F4B0036
:0426C900454E440036
:0426CD00434D440035
:0426D100414F4B002A
:0426D500414F4B0026
:0426D900414F4B0022
:0126DD0000FC
:0526DE004364653D00AE
:0226E3000000F5
:1026E50020436F74E92052464F2D42617369633A66
:1026F50020546573745F4750535F42545F313630E1
:0B2705003830342E626173200D0A0092
:102710005541525420434F4D313A31393230302CEB
:1027200020554152543220434F4D32203A313932F4
:062730003030200D0A000C
:1027360020464F53433D384D687A20696E74657262
:102746006E65207820504C4C203D3E2034384D6834
:062756007A20200D0A00AC
:10275C00436865636B2070726573656E6365204CAE
:10276C004344323131392061742040203078373481
:03277C000D0A0043
:10277F0053412C30202064697361626C6520617550
:10278F007468656E74696669636174696F6E0D0054
:10279F0053522C3443304233413842393435372089
:1027AF003D3E2053746172616469637449490D0041
:1027BF00204C696169736F6E204D6F64656C652085
:0E27CF00425420524E34312061766563200062
:1027DD00534E2C4D7942542D44423439203D3E20E8
:0E27ED00446576696365206E616D650D0A00B6
:1027FB00726573756C742042545F436F6E666967C4
:0E280B007572652829205374617465203D00A4
:1028190053522C3030313538333242364438372030
:0C2829003D3E2050435F41504D200D000B
:10283500496E697420493243322048617264776178
:0C2845007265203430304B687A0D0A00B8
:10285100464F53433D34384D485A2020504C4C206C
:0B28610061637469766520200D0A0099
:10286C0053542C323535203D3E20416C6C776179C8
:0B287C007320415420636465730D005D
:102887002D2D2D2020203D3E2046696E206D6F6442
:0B28970065206364652041540D0A00B9
:1028A2004250313D202020203B4250323D2020200A
:0A28B20020203B204541313D20006D
:1028BC00504F52542055534220484944205465727D
:0928CC006D696E616C200D0A00BB
:1028D5002041726D652049542055415254312026BE
:0928E5002055415254320D0A0045
:1028EE005472616D65204750532072656375652083
:0628FE003A20202020001A
:102904004465636F64616765205061727469656CC6
:06291400204F4B0D0A00EC
:10291A00496E6974204C434420323131392032786F
:05292A0031360D0A002A
:10292F002424240D20204154204D6F646520456ED2
:04293F007465720049
:1029430053582C3120203D3E20426F6E6465643D18
:03295300310D0043
:1029560053552C31392E32203D3E20626175647309
:032966000D0A0057
:10296900202F2039202050726F626C656D6F2021F5
:032979000D0A0044
:10297C004C41543A202020202020202020202020B0
:01298C00004A
:10298D005554433A20202020202020202020202094
:01299D000039
:10299E00425420436F6E66696775726174696F6E1B
:0129AE000028
:1029AF004574617065203A2031207375722039208B
:0129BF000017
:1029C00041726D6520496E74657272757074732002
:0129D0000006
:1029D1004574617065203A202E207375722039206C
:0129E10000F5
:1029E200417474656E74652047505320646174614C
:0129F20000E4
:1029F30042616420696E69742042542021212020A1
:012A030000D2
:102A0400496E697420425420636F6D706C657465FF
:012A140000C1
:102A1500496E6974204144432073757220454131E4
:012A250000B0
:102A2600546F2050435F585020636C652041504DD1
:012A3600009F
:102A370020546F205374617241646963744949205B
:012A4700008E
:102A4800203130302078203430203D2034736563C5
:012A5800007D
:102A5900496E69742054696D6572332034306D5341
:012A6900006C
:102A6A0053522C30303135383332423644383700FD
:102A7A00436865636B20446576696365204020007E
:102A8A0053522C34433042334138423934353700BB
:0F2A9A005374617261646963744949203A200082
:0F2AA900534D2C35203D3E20414E590D207200DB
:0E2AB80055415254312052656375203A20007A
:0E2AC60055415254312052656375203A20006C
:0E2AD400206973206E6F7420666F756E64004B
:0D2AE20020496E697420414443310D0A0003
:0D2AEF004438393532463346463731300021
:0D2AFC00534E2C4D7942542D444234390084
:0D2B0900536174656C6C697465733A20004B
:0D2B16003443304233413842393435370002
:0D2B23003030313538333242364438370017
:0C2B300053746172616469637449490068
:0B2B3C00202F203920204F4B0D0A00F5
:0B2B47004C617469747564653A2000ED
:0B2B520042313D2E2042323D2E20007B
:0A2B5D00627566666572323D200065
:0A2B670020666F756E64204F4B006E
:092B710032202048415244570073
:092B7A00415243484F533433002B
:092B83005374617465203D2000CB
:082B8C00206F6E204932430066
:082B94002447504747412C0083
:082B9C0053552C31392E320093
:072BA40050435F41504D005A
:072BAB0053542C32353500B4
:072BB2004C6F6E673A200032
:062BB9004C4F4E3A2000D3
:062BBF005574633A20008A
:052BC5002D2D2D0D0077
:052BCA002D2D2D0D0072
:052BCF0053582C3100F9
:052BD40053412C30000C
:052BD900534D2C3500F6
:042BDE002D2D2D006C
:020000040001F9
:06FFF800ACF7C2FFF8FFA8
:00000001FF
